:020000040000FA
:0400000019280000BB
:020008000528C9
:06000A00F0000308F600FF
:100010000A08F7000408F8008B1C0F280000830171
:100020007808840077088A0076088300F00E700E46
:1000300009008312031385018601870183160313C8
:1000400086018501FF30870006309F00831203136D
:10005000860185010030F300F400F500FF308600D2
:100060000708F200F51C3A2872184928F2184928A6
:10007000F510492872184328F21C4928061002304E
:100080008606F5144928F218492806140230860617
:10009000F514751D512872196028F2196028751120
:1000A000602872195A28F21D602806110830860649
:1000B00075156028F2196028061508308606751532
:1000C000F51D6828721A7728F21A7728F511772813
:1000D000721A7128F21E7728061220308606F5154E
:1000E0007728F21A7728061620308606F515751E31
:1000F0007F28721B8E28F21B8E2875128E28721B89
:100100008828F21F8E2806138030860675168E28E2
:10011000F21B8E28061780308606751630280000E0
:020120008F2826
:040122000034003471
:02400E007A3FF7
:00000001FF
